:020000040000FA
:020000000528D1
:0800080009008316FF2390009C
:1000100083128B0107309900831605108510051196
:100020008515051685168312831618309F008312D6
:100030000511051085100030AA000130AB00FF301B
:10004000AC0085194F28851A4F2805148514851D85
:100050003B28851E3B281E08A6002B08A700CB20A6
:10006000C830C120C830C12005148514C830C12053
:100070000510851030280D309F000130C1209F14DD
:100080009F1840281E08A200A20A05150130C120B1
:100090000000A20B482805111230C120272800308B
:1000A000A8000030A90083162A089B001C141A0817
:1000B000A500831283162B089B001C141A08AC00A1
:1000C0008312A508031D68280130A30005146E28BB
:1000D0000130A5002C08A300A303851464002308A5
:1000E000A20005150130C1202308A2000000A20BC8
:1000F000762805111230C120A808031DAA28A908D6
:10010000031D9428851985288828851A6E288E282D
:10011000A508031DAA280130A800AA28A5080319CC
:1001200094280130A9009428A30B9B28A30AA508B2
:10013000031D9E286E28051485146E280030A50026
:100140002508A6002A08A700CB200514851000303A
:10015000A9006E28A30A2308A4002C082402031D6A
:100160009B28A303A508031D6E280130A5002508C0
:10017000A6002A08A700CB20051085140030A8008F
:100180006E28A000C830A10000000000A10BC42808
:10019000A00BC2280800831627089B0026089A0097
:1001A0001C158B1355309D00AA309D009C141C110A
:0A01B0008B179C18D9288312080051
:02400E00C43FAD
:00000001FF
